:020000002428B2
:08000800C428F2017008F300A6
:100010007108031D0E28FF30F20019287108F00244
:10002000031C1628F20A7008F3000E280310720849
:100030000319031408001830A6000830A500A50B0A
:100040001F28A60B1D280034831207309F00900143
:100050009016101683165F309200D53081000C1474
:100060008C10E0308B0000308600FF30850083125A
:10007000101097019715171512149210121186017E
:10008000C001C901CA01CB01C201C301C401C5013C
:10009000C101A101A001AE01CC01703081001F306F
:1000A0008F008E016430A700A801A901AA01A40154
:1000B0008B1383160A309B001C141A088312AB00A2
:1000C0008B178B1383160B309B001C141A0883129A
:1000D000AC008B178B1383160C309B001C141A0872
:1000E0008312AF008B178B1383160D309B001C14EB
:1000F0001A088312B0008B178B1383160E309B00E7
:100100001C141A088312B1008B178B13831610303E
:100110009B001C141A088312CE008B178B138316B6
:1001200011309B001C141A088312CF008B178B13FD
:10013000831612309B001C141A088312CD008B17F3
:100140008B13831613309B001C141A088312B20001
:100150008B178B13831614309B001C141A08831200
:10016000AD008B173008033A0319BE283008023A55
:100170000319BC287E22BF288622BF288E220C307D
:10018000E200E30128249429C700030EC8000B19DC
:10019000CC280C18D628DD280B1170308100521E97
:1001A000E223CA0AA70BDD28E220DD281010121175
:1001B0000C101F308F008E018611480E8300C70E71
:1001C000470E09006430A7004108003A0319EA28E5
:1001D000C101EB2841142D080319F7282E08031933
:1001E000F728281CF5281215F72812118611A80ADD
:1001F00028083C3A0319FD286A29D21B0429D21980
:100200000429D215E10BD211A801A90A2D0803195E
:1002100027292E08031D18292A082B06031911293E
:10022000272929082C06031916292729AE0112159A
:10023000AE0A2F082E02031C222903102E082F06B7
:10024000031D242900002729AE0112118611CB0AB3
:100250004B080B3A03192D292F29CB01A80A29088D
:100260003C3A031934296A2931080319392912152E
:100270001014D21B3F29521A3F29D2192824A90150
:10028000AA0A2D0803194E292C08031D4E292A08F5
:100290002B06031D4E29AE011215AE0A2A08033A99
:1002A000031957292A080F3A031957295929521EA9
:1002B00028242A08183A03195E296A29A801A901E5
:1002C000AA012D0803196A292B08031D6A29AE010A
:1002D0001215AE0A401C7B2108002308A200A20DC3
:1002E000A20DA20DA20D2208F039460786001B20A0
:1002F0001B201B2008002908F00020182C08F00003
:100300000A30F10005207308C5007208C4002A08ED
:10031000F00020182B08F0000A30F10005207308C7
:10032000C3007208C20008004408A3000130C600E0
:100330006D214208A3002308003A0319A1290330C4
:10034000A2290730C6006D214508A3000030C60071
:100350006D214308A3000230C6006D21521AB62950
:10036000D21BB629D219B629411CBC290430C600BB
:100370006D210530C6006D212D08003A0319C329EF
:100380000630C6006D2105080F39A200A001A21891
:1003900020142208033A0319EC292208053A03190C
:1003A0001D2A2208093A03192A2A2208063A0319A3
:1003B000372A22080A3A0319442A2208083A03195C
:1003C000F8292208023A03191A2A2208013A0319C5
:1003D0001A2AA101CA019429A001C8304A02031CAB
:1003E000F62903104A08C83A031D962A00009429EA
:1003F0002118942921142D08003A0319042AAD016B
:10040000AE0186111211052A2D148B131430831698
:100410009B0083122D0883169A001C1555309D00F1
:10042000AA309D009C141C1183128C1F152A8C135A
:100430008B1794297B21A101942921189429211437
:10044000AA0A2A08183A0319272A7B219429AA0103
:100450007B219429211894292114A90A29083C3ABE
:100460000319342A7B219429A9017B21942921187D
:1004700094292114AB0A2B08183A0319412A7B212D
:10048000502AAB017B21502A211894292114AC0A4F
:100490002C083C3A03194E2A7B21502AAC017B21BF
:1004A0008B130A3083169B0083122B0883169A0045
:1004B0001C1555309D00AA309D009C141C11831200
:1004C0008C1F602A8C138B178B130B3083169B00A9
:1004D00083122C0883169A001C1555309D00AA30F3
:1004E0009D009C141C1183128C1F742A8C138B1773
:1004F0009429A4011219241512110800792202303E
:10050000950097161716241912150800792206303F
:100510009500971617122419121508007922343005
:10052000950097121716241912150800CA01BD2349
:1005300040144508A3000030C6006D214408A30004
:100540000130C6006D214308A3000730C6006D21AD
:100550004208A3000330C6006D2105080F39A20030
:100560002208033A0319992A2208023A0319332B65
:100570002208083A0319402B2208043A03198D2B4C
:100580002208013A0319C72AA101CA01992A643035
:100590004A02031CD02A03104A08643A031DD22AD7
:1005A0000000992A2118992A40108B130C308316C9
:1005B0009B0083122F0883169A001C1555309D004E
:1005C000AA309D009C141C1183128C1FE52A8C13E9
:1005D0008B178B130D3083169B0083123008831604
:1005E0009A001C1555309D00AA309D009C141C11CA
:1005F00083128C1FF92A8C138B178B130E308316E2
:100600009B008312310883169A001C1555309D00FB
:10061000AA309D009C141C1183128C1F0D2B8C136F
:100620008B178B13103083169B0083124E08831692
:100630009A001C1555309D00AA309D009C141C1179
:1006400083128C1F212B8C138B173008033A03194C
:10065000312B3008023A03192F2B7E22942986224F
:1006600094298E2294292118992A2114CC0A4C0805
:10067000320603193D2BBD23992ACC01BD23992AAB
:100680002118992A21144C08003A0319542B4C08BC
:10069000013A03195B2B4C08023A0319622B4C08F0
:1006A000033A0319692B992AAF0A2F085B3A0319F9
:1006B000702BBD23992AB00A3008043A0319702B15
:1006C000BD23992AB10A3108023A0319702BBD23C0
:1006D000992ACE0A4E08023A0319702BBD23992A93
:1006E0004C08003A0319802B4C08013A0319832B5C
:1006F0004C08023A0319862B4C08033A0319892B3C
:100700005A30AF008B2B0330B0008B2B0130B1007F
:100710008B2B0130CE00BD23992A2118992A211450
:100720004C08003A0319A12B4C08013A0319A82BD5
:100730004C08023A0319AF2B4C08033A0319B52BA6
:10074000992A2F08013A0319992AAF03BD23992A40
:100750003008013A0319992AB003BD23992A3108B8
:100760000319992AB103BD23992A4E080319992A1E
:10077000CE03BD23992ABD23992A4C08003A0319B8
:10078000CD2B4C08013A0319D02B4C08023A03191F
:10079000D32B4C08033A0319D62B2F08F000D82B83
:1007A0003008F000D82B3108F000D82B4E08F000AC
:1007B0000A30F10005207308C5007208C4004C0817
:1007C000C2000800D219272CD21F262C521B272C1E
:1007D0004E0803191F2C4F080319092C4F08013A22
:1007E0000319F32B1F2C53084D075718013EA20085
:1007F00017302202031C012C03102208173A031D94
:10080000052C00002208AA00212C18302202AA0080
:10081000212C4D085718013EA20022085302031C48
:10082000152C22085302AA00212C5308183ED3008D
:1008300022085302AA005308183CD300212C530865
:10084000AA005508A900A8015217272C392408002E
:100850000530E1006430D000D101D201D301D501CF
:10086000D701D801D901DB01DE01E001FF30DF0053
:100870000800051E3C2C552C0C30E200E301521CF4
:100880004E2C51080319602C11305102031C4A2CC4
:10089000D2144B2CD210D101DF0A612CD0030319E2
:1008A000522C602C5214D101602CE30F5B2CE20B14
:1008B0005B2C000052166430D000521C602CD10A10
:1008C00008005F08113A0319662C682CD2185714D7
:1008D0005F08123A03196D2C6F2CD21857105F085D
:1008E000143A0319742C782CD218782C2A24602CF2
:1008F0005F08153A0319532D5F08163A03195A2D4C
:100900005F08173A0319612D5F08183A0319682D1B
:100910005F08193A03196F2D5F081A3A0319762DEB
:100920005F081B3A03197D2D5F081C3A0319482EF6
:100930005F081D3A0319842D5F081E3A03198B2D99
:100940005F081F3A0319922D5F08203A0319992D69
:100950005F08213A0319A02D5F08223A0319A72D39
:100960005F08233A0319482E5F08243A0319AE2D75
:100970005F08253A0319B52D5F08263A0319BC2DE7
:100980005F08273A0319C32D5F08283A0319CA2DB7
:100990005F08293A0319D12D5F082A3A0319D82D87
:1009A0005F082B3A0319DF2D5F082C3A0319E62D57
:1009B0005F082D3A0319ED2D5F082E3A0319F42D27
:1009C0005F082F3A0319FB2D5F08303A0319022EF6
:1009D0005F08313A0319092E5F08323A0319102EC5
:1009E0005F08333A0319172E5F08343A03191E2E95
:1009F0005F08353A0319252E5F08363A03192C2E65
:100A00005F08373A0319332E5F08383A03193A2E34
:100A10005F08393A0319412E5F083A3A0319482E04
:100A200059305502031C192D03105508593A031D5E
:100A3000762C000023305302031C232D031053088F
:100A4000233A031D762C000031305902031C2D2D52
:100A500003105908313A031D762C000012305B0256
:100A6000031C372D03105B08123A031D762C00007F
:100A700007305802031C412D03105808073A031D84
:100A8000762C000099305E02031C4B2D03105E088B
:100A9000993A031D762C00005F083B3A0319512D4B
:100AA000602CD217602CD21C602CE00A5508013E45
:100AB000D500602CD21C602CE00A5508023ED500FF
:100AC000602CD21C602CE00A5508043ED500602C36
:100AD000D21C602CE00A5508083ED500602CD21CC0
:100AE000602CE00A55080A3ED500602CD21C602C10
:100AF000E00A5508143ED500602CD21C602CE00A98
:100B00005508283ED500602CD21C602CE00A530802
:100B1000013ED300602CD21C602CE00A5308023E38
:100B2000D300602CD21C602CE00A5308043ED30092
:100B3000602CD21C602CE00A5308083ED300602CC5
:100B4000D21C602CE00A53080A3ED300602CD21C51
:100B5000602CE00A5308143ED300602CD21C602C99
:100B6000E00A5908013ED900602CD21C602CE00A32
:100B70005908023ED900602CD21C602CE00A5908AA
:100B8000043ED900602CD21C602CE00A5908083EB3
:100B9000D900602CD21C602CE00A59080A3ED9000A
:100BA000602CD21C602CE00A5908143ED900602C3D
:100BB000D21C602CE00A5808013ED800602CD21CE0
:100BC000602CE00A5808023ED800602CD21C602C31
:100BD000E00A5808043ED800602CD21C602CE00AC1
:100BE0005B08013EDB00602CD21C602CE00A5B0835
:100BF000023EDB00602CD21C602CE00A5B08043E45
:100C0000DB00602CD21C602CE00A5B08083EDB0095
:100C1000602CD21C602CE00A5B080A3EDB00602CD2
:100C2000D21C602CE00A5E08013EDE00602CD21C63
:100C3000602CE00A5E08023EDE00602CD21C602CB4
:100C4000E00A5E08043EDE00602CD21C602CE00A44
:100C50005E08083EDE00602CD21C602CE00A5E08B4
:100C60000A3EDE00602CD21C602CE00A5E08143EB6
:100C7000DE00602CD21C602CE00A5E08283EDE00FC
:100C8000602CD21C602CE00A5E08503EDE00602C16
:100C900060184E2ED2182A24E001602CD21C2A247F
:040CA000E001602CE3
:100D00004400690065007300650073002000500016
:100D100072006F006700720061006D006D002000BE
:100D2000690073007400200075007200680065009F
:100D30006200650072007200650063006800740064
:100D40006C006900630068002000670065007300A4
:100D5000630068007500650074007A00740020006C
:100D6000210041006C006C0065002000520065000D
:100D70006300680074006500200056006F00720078
:100D800062006500680061006C00740065006E0020
:100D900020002100450069006E00730061007400AE
:100DA0007A00200061007500730073006300680022
:100DB0006C0069006500730073006C0069006300DB
:100DC0006800200061007500660020006500690071
:100DD000670065006E006500200047006500660042
:100DE000610068007200200021004B00650069006E
:100DF0006E00650020004800610066007400750008
:100E00006E0067002C0020006500670061006C0028
:100E100020006100750073002000770065006C0001
:100E20006300680065006D002000470072007500D7
:100E30006E00640020002100460072006500690019
:100E400020006600FC007200200070007200690043
:100E5000760061007400650020004E00750074008B
:100E60007A0075006E0067002E004B006F006D0069
:100E70006D00650072007A00690065006C006C000E
:100E8000650020004E00750074007A0075006E0049
:100E9000670020006E007500720020006D00690080
:100EA000740020007300630068007200690066002F
:100EB00074006C0069006300680065007200200027
:100EC000470065006E00650068006D0069006700FE
:100ED00075006E0067002000210045002E004D00C7
:100EE000750065006C006C006500720050006F00BA
:100EF0007300740066006100630068002000370022
:100F00003000310033003700310044002D0038003C
:100F1000310033003100330020004D0075006500C2
:0A0F20006E006300680065006E00BB
:02400E00613F10
:0C42140007001E000F0001000100000068
:0A4220000000000001000300000090
:00000001FF
